:101FA6002020202020200D0A002A56455253494F52
:101FB6004E3A20522D4441532056322E320D0A00FD
:101FC6002A4D4553534147453A2053656C6674651F
:101FD6007374207061737365640D0A002A57415249
:101FE6004E494E473A2053656C6674657374206695
:101FF60061696C65640D0A002A52454144590D0A0F
:0120060000D9
:101CC100D2AF1228D912298F12000E12284F122AD0
:101CD100501229E8122A1C7BFF7A1F79A61200C92B
:101CE1007BFF7A1F79AF1200C91224FA50127BFFD1
:101CF1007A1F79C61200C97F017D0112263380093E
:101D01007BFF7A1F79E21200C9121EDC906C99E008
:101D1100FF1224881226DB1221CB906C9AE0FEA3DD
:101D2100E0FF1223C87BFF7A1F79FE1200C9122837
:021D3100BF22CF
:03000B000220C709
:1020C700C0E0C0F0C083C082C0D075D008E550F52D
:1020D7008CE551F58AD55509906C90E0F555122796
:1020E700AED5541B906C90E0F5540553E553700240
:1020F7000552E55345527007E55A6003755A05E5E1
:102107005A64046009121401121C4E121A22D0D00C
:09211700D082D083D0F0D0E03278
:1023C800E4FCFDFB7AC079A8F81204ED7BE07A2ED4
:1023D80079007800122341C3E49FF551E49EF5503B
:1023E800906C90E0F555F554E4F552F553E58954B1
:1023F800F04401F589758CFF758AFFC2B9D2A9D25C
:022408008C2224
:0C29BA00906C90E0F554E4F552F55322C7
:1021CB00E5C520E3FB75C50775C50FE5C530E4FB19
:1021DB00AFC6EF75F004A4FFAEF0E5C5C4131354FE
:1021EB00037C002FF52DEC3EF52CE4F52BE52B2590
:1021FB00E024ACF8A62C08A62DE52D2528F528E51E
:10220B002C3527F527052BE52BB40AE1E4F52A221B
:10140100C0D075D008301B03021502E5C520E3FBEF
:10141100E4F5C575C508F533753401E53364087025
:10142100030214E4E5C530E4FB85C62985C52EE534
:10143100336407600EE5C520E3FBE53304F5C544DD
:1014410008F5C5906C8FE0553470030214D9AF29AB
:1014510012259DAF2E12259DE533B4061BE5297596
:10146100F004A4FFAEF0E52EC4131354037C002F47
:10147100F532EC3EF5318060E5336407705AE52AB8
:1014810025E024ADF8C3E52896F528E5271896F55B
:1014910027E52975F004A4FFAEF0E52EC41313541B
:1014A100037C002FF536EC3EF535E52A25E024AC2A
:1014B100F8A63508A636E5362528F528E535352779
:1014C100F527FEAF287D0A1204368E258F26052AC0
:1014D100E52AB40A03E4F52A0533E53425E0F534B9
:1014E10002141C30171BE4A2C492E4A2C592E5A227
:1014F1009692E6A29792E7255AC4F52FAF2F1225AF
:041501009DD0D02287
:101D3300C0D075D008301765906C99E0FD7C009099
:101D43006CA1E0FB24FFFFE434FFFE120422EF2426
:101D530001FFE43EFEC3E51F9FF51FE51E9EF51E32
:101D63008B30E5306021E51EF583E51FF582E0C485
:101D730054F0255AC4F0906C99E0251FF51FE43503
:101D83001EF51E153080DB906C99E024FFFFE434D0
:101D9300FFFEC3E51F9FF51FE51E9EF51ED0D02253
:10297F0053544F52452069732066756C6C0D0A00D5
:0D29AD00E4F563F564F565C21B1224C12238
:101C4E00C0D075D008E55A6067201B641229494040
:101C5E005F906C99E025E0906CDBF0906CDBE060BF
:101C6E004F20194C1225D18F6212002E0564E564A7
:101C7E00700205637004E5636480702CF563F5648F
:101C8E000565E565B40C147BFF7A29797F1200C9CE
:101C9E007F037D01122633D21B8015122936E5658E
:101CAE0020E0051224C18008906CDBE014F080ABBC
:031CBE00D0D02261
:10240A00464C494748545F4C61756E63680D0A0033
:10241A00464C494748545F456A6563745061726126
:10242A006368757465310D0A00464C494748545F24
:10243A00456A656374506172616368757465320DCB
:02244A000A0086
:1026DB00E4906D2BF0A3F0906D27120582000000A3
:1026EB000074FF906D23F0A3F0E4906D2DF0F55B7B
:0526FB00F55AC21C228B
:1027F000C0D075D0087BFF7A24790A1200C9755AB7
:1028000001C2901229AD7F027D01122633D0D02261
:10274800C0D075D0087BFF7A24791A1200C9C291CB
:10275800E5532401906D26F0E43552906D25F0D0B4
:02276800D0227D
:10276A00C0D075D0087BFF7A2479331200C9C2928F
:10277A00E5532401906D26F0E43552906D25F0D092
:02278A00D0225B
:10160700C0D075D008301C3330C63F30C73CC21C31
:10161700906D33E0FF60077D04122633802C906DB8
:1016270032E0FF64036004EFB404077D041226333D
:1016370080187F017D01122633800F30C60320C733
:10164700097F027D04122633D21C30131EA2943068
:101657001401B34016C21E1229BA906C8DE0FEA386
:10166700E0FF1226051227F00216F92018030216CA
:10167700F9906C8BE0FEA3E0FFC3E5469FFFE545CD
:101687009EFED3E5329FE5319E4016D21E906D2710
:1016970012058200000000E4906D2BF01229BA8039
:1016A70051C21E906D27E0F8A3E0F9A3E0FAA3E08A
:1016B700FBC3E5329546FFE5319545FE3395E0FDE1
:1016C700FCEB2FFFEA3EFEE93DFDE83CFC906D2771
:1016D700120576906CA1E0FF906D2BE004F06F701F
:1016E70011906C94E0FEA3E0FF1226051227F0127A
:0516F7001D33D0D022DC
:101B5300C0D075D008906D27E0F8A3E0F9A3E0FAB0
:101B6300A3E0FBC3E5329546FFE5319545FE33958A
:101B7300E0FDFCEB2FFFEA3EFEE93DFDE83CFC9077
:101B83006D271205763016337F007E007D007C00C2
:101B9300906D27E0F8A3E0F9A3E0FAA3E0FBD312EA
:101BA300053C4017906C8AE0FFD3E5539FE55294C0
:101BB300004008122748755A028015301512906CA0
:101BC3009FE065537002E5527006122748755A0A62
:031BD300D0D0224D
:101DA300C0D075D008906D25E0FEA3E065537003A5
:101DB300E5526E7002D291301637906C97E0FEA315
:101DC300E0FFC3E5489FFFE5479EFEC3E5269FE589
:101DD300259E5007E4906D2CF08016906CB2E0FFC6
:101DE300906D2CE004F06F700812276A755A038017
:101DF30015301512906CA0E065537002E552700621
:091E030012276A755A0BD0D02297
:10286C00C0D075D008906D25E0FEA3E065537003D1
:0C287C00E5526E7004D291D292D0D022AE
:101A2200C0D075D008E55A6071E4F556755901E5E4
:101A32005664086065E55625E024A2F582E4346C1C
:101A4200F583E0FEA3E08E57F558F47003E557F4F2
:101A5200603EE55B55597015E55365587004E552D3
:101A620065577009E559425BAF56122267E55B552F
:101A720059601DE5582401FFE43557FEEF655370A8
:101A820003EE6552700AE559F4525BAF561222B268
:101A92000556E55925E0F5598095E55A1460161466
:101AA200601814601A24F96011146013240B701268
:101AB200121607800D121B538008121DA3800312F9
:051AC200286CD0D022C9
:10248800CBEFCBEBFD7C007E407F00120436CDEB1A
:10249800CD7C001204228E1A8F1B74002FF582EE59
:1024A800342CAF82F5188F197E2C7F008E1C8F1D5F
:0924B8008E1E8F1FD219C21A22D8
:10259D00C219051FE51FAC1E7002051E14F5828CB5
:1025AD0083EFF0E51F65197004E51E65187006755B
:1025BD001E2C751F00E51F651D7004E51E651C7042
:0425CD0002D21A22FA
:1025D100C21A051DE51DAE1C7002051C14F5828E84
:1025E10083E0FFE51D65197004E51C65187006752B
:1025F1001C2C751D00E51F651D7004E51E651C7012
:0426010002D21922C6
:10260500C3E51F9FF51DE51E9EF51CC3E51D940042
:10261500E51C942C400BD3E51D9519E51C95184038
:0E2625000CE51B251DF51DE51A351CF51C22C4
:10196700257320256275202562752025752025752C
:101977002025627520256275202563202562752044
:1019870025632025632025630D0A00632069676EA0
:10199700202575202575202575202575202575207E
:1019A70025752025752025750D0A006320786D693A
:1019B7007420257520256275202562750D0A002A79
:1019C70056455253494F4E3A20522D4441532056C3
:1019D700322E320D0A0063210063207264617300A6
:1019E700632069676E006320786D697400633F0048
:1019F700630063200072657365740070660070642D
:101A0700002A4552524F523A20556E6B6E6F776ED1
:0B1A170020636F6D6D616E640D0A00AE
:062A1C00E4F56AC21D2270
:100AD600906CE0EBF0A3EAF0A3E9F03013133014C6
:100AE60008906CFD7401F0800D906CFD7402F0802E
:100AF60005E4906CFDF0906CE0E0FBA3E0FAA3E067
:100B0600F91203BA643F6003020BAE906CE3E0F99E
:100B1600A3E0FAA3E0906CB6C9F0A3EAF0A3E9F06B
:100B2600906C90E0906CB9F0906C8FE0906CBAF09D
:100B3600906C8BE0FFA3E0906CBBCFF0A3EFF0903E
:100B46006C97E0FFA3E0906CBDCFF0A3EFF0906C44
:100B56009FE0906CBFF0906CA0E0906CC0F03017F6
:100B6600047F3180027F30906CC1EFF0906CFDE025
:100B7600906CC2F03018047F3180027F30906CC3D5
:100B8600EFF03016047F3180027F30906CC4EFF0B6
:100B96003015047F3180027F30906CC5EFF07BFF0B
:100BA6007A1979671200C922906CE0E0FBA3E0FA9B
:100BB600A3E0F91203BAFF122921500C906CE1E46C
:100BC60075F0011204C180E0E4906CFCF0906CE0DA
:100BD600E0FBA3E0FAA3E0F91216FC906CFCE0251A
:100BE600E024E6F582E4346CF583EEF0A3EFF090B2
:100BF6006CE0E0FBA3E475F0011204D7A9F0FA1249
:100C060003BAFF12292150E7906CFCE004F0E0B42F
:100C16000BBB906CE7E0906C90F0906CE9E0906C08
:100C26008FF0906CEAE0FFA3E0906C8BCFF0A3EF1F
:100C3600F0906CECE0FFA3E0906C97CFF0A3EFF0A0
:100C4600906CEFE0906C9FF0906CF1E0906CA0F0EF
:100C5600906CF2E0FEA3E0FFEE4F24FF9217A3E0B4
:100C6600FEA3E0FFEE4F24FF9213EF64014E7003E4
:100C7600D38001C39214906CF6E0FEA3E0FFEE4F22
:100C860024FF9218A3E0FEA3E0FFEE4F24FF921686
:0D0C9600A3E0FEA3E0FFEE4F24FF92152225
:10150500906CE0EBF0A3EAF0A3E9F01203BA643FB4
:10151500600302159C7BFF7A197992906CA2E0FF1B
:10152500A3E0906CB6CFF0A3EFF0906CA4E0FFA31E
:10153500E0906CB8CFF0A3EFF0906CA6E0FFA3E0CD
:10154500906CBACFF0A3EFF0906CA8E0FFA3E09009
:101555006CBCCFF0A3EFF0906CAAE0FFA3E0906C19
:10156500BECFF0A3EFF0906CACE0FFA3E0906CC0B1
:10157500CFF0A3EFF0906CAEE0FFA3E0906CC2CF8C
:10158500F0A3EFF0906CB0E0FFA3E0906CC4CFF057
:10159500A3EFF01200C922906CE0E0FBA3E0FAA3F0
:1015A500E0F91203BAFF122921500C906CE1E475A1
:1015B500F0011204C180E0E4906CE3F0906CE0E08F
:1015C500FBA3E0FAA3E0F91216FC906CE3E025E03A
:1015D50024A2F582E4346CF583EEF0A3EFF0906C71
:1015E500E0E0FBA3E475F0011204D7A9F0FA1203B9
:1015F500BAFF12292150E7906CE3E004F0E0B4084B
:02160500BB2206
:1018A300906CE0EBF0A3EAF0A3E9F01203BAB43FC3
:1018B300297BFF7A1979B2906C91E0FFA3E0906CD9
:1018C300B6CFF0A3EFF0906C9EE0906CB8F0906C04
:1018D30093E0906CB9F01200C922906CE0E0FBA396
:1018E300E0FAA3E0F91203BAFF122921500C906C1D
:1018F300E1E475F0011204C180E0E4906CE9F0903A
:101903006CE0E0FBA3E0FAA3E0F91216FC906CE9AB
:10191300E025E024E3F582E4346CF583EEF0A3EFF5
:10192300F0906CE0E0FBA3E475F0011204D7A9F09A
:10193300FA1203BAFF12292150E7906CE9E004F090
:10194300E0B403BB906CE3E0FFA3E0906C91CFF0B5
:10195300A3EFF0906CE6E0906C9EF0906CE8E09062
:041963006C93F0226F
:1006F9007B017A6C794C7D20122888906CE3EBF0B1
:10070900A3EAF0A3E9F04A70047F0180027F009018
:100719006CF0EFF0605F7B017A6C794B1212F3C8D1
:10072900ECC8C9EDC9CAEECACBEFCB906C9CE0FE10
:10073900A3E0FFE4FCFD1204EDC8ECC8C9EDC9CA89
:10074900EECACBEFCB906C8DE0FEA3E0FFE4FCFD9D
:10075900EB2FFFEA3EFEED39FDEC38FC906CE6121A
:100769000576906C9CE0FEA3E0FFE4FCFD906CEA4A
:1007790012057680767B017A6C794B1212F3C8ECFC
:10078900C8C9EDC9CAEECACBEFCB906C99E0FFE4BA
:10079900FCFDFE1204EDC8ECC8C9EDC9CAEECACB0E
:1007A900EFCB906C8DE0FEA3E0FFE4FCFDEB2FFFA7
:1007B900EA3EFEED39FDEC38FC906CE612057690C8
:1007C9006CE3E0FBA3E0FAA3E0F91212F3C8ECC86A
:1007D900C9EDC9CAEECACBEFCB906C99E0FFE4FC36
:1007E900FDFE1204ED906CEA120576906CE6E0FCD1
:1007F900A3E0FDA3E0FEA3E0FF780F1205638F6578
:10080900906CE6E0FCA3E0FDA3E0FEA3E0FFEE545C
:100819007FFEE48E638F64122936906CF0E06009E4
:10082900E4906CEEF0A3F0800B120026906CEEEED3
:10083900F0A3EFF0E4906CE0F0A3F0906CE0E0FE40
:10084900A3E0FFE4FCFD906CEAE0F8A3E0F9A3E083
:10085900FAA3E0FBC3120552606C1229C6906CE240
:10086900EFF0906CF0E06014906CE2E0FF906CEFB8
:10087900E02FF0906CEEE03400F08018906CEEE020
:10088900FEA3E0FF906CE2E0FD121BD6906CEEEE49
:10089900F0A3EFF0906CE2E0FF1200030564E56459
:1008A900700205637004E56364807009F563F5649B
:1008B9000565122936906CE1E004F07006906CE051
:1008C900E004F0020844906CF0E07013906CEEE0E4
:1008D900FEA3E0FF122A15906CEEEEF0A3EFF09064
:1008E9006CEEE0FF120003906CEFE0FF12000322B0
:042A400012278C22AB
:0A29DE007BFF7A1979C61200C922A6
:100CA300906CE374FFF0A37419F0A374DDF0A3E474
:100CB300F0A37402F07B017A6C794A121E75EF700F
:100CC3000412100722906CE374FFF0A37419F0A3CD
:100CD30074E0F0A3E4F0A37406F07B017A6C794A24
:100CE300121E75EF7018906CE374FFF0A37419F083
:100CF300A374E0F07B017A6C7950120AD622906CCF
:100D0300E374FFF0A37419F0A374E7F0A3E4F0A372
:100D13007405F07B017A6C794A121E75EF700A7BB9
:100D2300017A6C794F12150522906CE374FFF0A3DE
:100D33007419F0A374EDF0A3E4F0A37406F07B013F
:100D43007A6C794A121E75EF700A7B017A6C7950BE
:100D53001218A322906CE374FFF0A37419F0A37428
:100D6300F4F0A3E4F0A37402F07B017A6C794A12E5
:100D73001E75EF7018906CE374FFF0A37419F0A361
:100D830074F7F07B017A6C794B120AD622906CE3EC
:100D930074FFF0A37419F0A374F9F0A3E4F0A3743F
:100DA30002F07B017A6C794A121E75EF7018906C11
:100DB300E374FFF0A37419F0A374F7F07B017A6C6A
:100DC300794B120AD622906C4AE0B464041206F9F5
:100DD30022906CE374FFF0A37419F0A374FCF0A3E6
:100DE300E4F0A37405F07B017A6C794A121E75EF67
:100DF3007004122A4022906CE374FFF0A3741AF07B
:100E0300A37402F0A3E4F0A37402F07B017A6C797B
:100E13004A121E75EF700D7B017A6C794E1216FC27
:100E2300122A5322906CE374FFF0A3741AF0A37494
:100E330005F0A3E4F0A37402F07B017A6C794A1203
:100E43001E75EF700D7B017A6C794E1216FC122A17
:100E53005622906C4AE0B476041229DE22906C4A42
:0D0E6300E060097BFF7A1A79081200C922AD
:1028BF00101D0280FB755A047F017D011226337FA4
:0A28CF001E12295C120CA380E72200
:10253300C0D0EF20E72CEF640A6027EF640D601131
:10254300744A256AF582E4346CF583EFF0056A80FA
:1025530011744A256AF582E4346CF583E4F0D21DE4
:05256300F56AD0D02252
:101E0C002A4D4553534147453A2053746F72696EBE
:101E1C006720706172616D657465727320696E20E4
:101E2C00464C4153480D0A002A4D455353414745F2
:101E3C003A2046696E69736865642073746F7269C1
:101E4C006E670D0A00000001C001C802000C0014EE
:101E5C000100193C03FFFFFFFFFFFFFFFFFFFFFF28
:091E6C00FFFFFFFFFF0000000072
:0A29E80075661E75675112118E22EC
:10118E00901E51E49324FF9213A3E49324FF921430
:10119E00A3E49324FF9218A3E493906C8FF0901E17
:1011AE0055E49324FF9217E4906C99F07F80EF60E2
:1011BE0014906C8FE05F6007906C99E02402F0EF62
:1011CE00C313FF80E9301706906C99E004F0901E6F
:1011DE0056E493906C90F0901E57E493906C96F0BA
:1011EE00901E58E493FF740193906C8BCFF0A3EF95
:1011FE00F0901E5AE493FF740193906C97CFF0A376
:10120E00EFF0906C90E0FBFD7C007E037FE8120413
:10121E0036906C9AEEF0A3EFF0906C99E0FA8BF0AA
:10122E00A4FF906C9CE5F0F0A3EFF0EB1313543F8A
:10123E00906CA1F0FB906CB2F0901E5CE49324FFD6
:10124E009216A3E49324FF9215A3E493906C9FF05F
:10125E00901E5FE493906CA0F0901E60E493906CEF
:10126E008AF0906C96E0FF7E00906C9CE0FCA3E010
:10127E00FD120422906C8DEEF0A3EFF0EBFF7E00DA
:10128E00EAFD7C00120422E02F906C95F0906C8D9C
:10129E00E03E906C94F0E4FFEF25E02461F582E4EB
:1012AE00341EF583E493FC740193FDEF25E024A234
:1012BE00F582E4346CF583ECF0A3EDF00FEFB40897
:1012CE00D7901E71E493FF740193906C91CFF0A3AD
:1012DE00EFF0901E73E493906C9EF0901E74E49366
:0512EE00906C93F0225A
:10100700A213E433856782856683F0A214E433A3D1
:10101700F0A218E433856782856683A3A3F0906CFA
:101027008FE0856782856683A3A3A3F0A217E433C5
:10103700FFE5672404F582E43566F583EFF0906CED
:1010470090E0FFE5672405F582E43566F583EFF068
:10105700906C96E0FFE5672406F582E43566F58334
:10106700EFF0906C8BE0FEA3E0FFE5672407F582C5
:10107700E43566F583EEF0A3EFF0906C97E0FEA3FE
:10108700E0FFE5672409F582E43566F583EEF0A312
:10109700EFF0A216E433FFE567240BF582E435662B
:1010A700F583EFF0A215E433FFE567240CF582E43E
:1010B7003566F583EFF0906C9FE0FFE567240DF54B
:1010C70082E43566F583EFF0906CA0E0FFE56724D6
:1010D7000EF582E43566F583EFF0906C8AE0FFE564
:1010E70067240FF582E43566F583EFF0E4906CE052
:1010F700F0906CE0E0FF6408603BEF25E024A2F588
:1011070082E4346CF583E0FEA3E0FFE5672410F585
:1011170082E43566F583C083C082906CE0E0D082BC
:10112700D08375F0021205B3EEF0A3EFF0906CE0F8
:10113700E004F080BC906C91E0FEA3E0FFE567243B
:1011470020F582E43566F583EEF0A3EFF0906C9E10
:10115700E0FFE5672422F582E43566F583EFF0903A
:101167006C93E0FFE5672423F582E43566F583EFAA
:10117700F07BFF7A1E790C1200C91225687BFF7A73
:071187001E79341200C92299
:101EDC00E5C520E3FB75C50675C50EE5C530E4FB0D
:101EEC00AFC6EF75F004A4FFE5C5C4131354037C0F
:101EFC00002FFFEC35F0CF2401F542E43FF541F51E
:101F0C0045854246E5C520E3FB75C50775C50FE55C
:101F1C00C530E4FBAFC6EF75F004A4FFAEF0E5C529
:101F2C00C4131354037C002FF544EC3EF543F547E2
:061F3C00854448D21E227C
:1027AE00301E1D854145854246E5322401F542E441
:1027BE003531F54185434785444885254385264473
:0127CE0022E8
:1028D900C21F43878075985AE589540F4420F589AA
:0A28E900758DFFD28ED2BCD2AC2256
:0300230002268929
:10268900C0E0C0F0C083C082C0D075D010309807B8
:10269900AF99C298122533309904C299D21FD0D06C
:0926A900D082D083D0F0D0E032E1
:080003008F99301FFDC21F227E
:082A06008F99301FFDC21F2251
:1026B200E5C520E3FB8FC5EF4408F5C5E5C530E469
:1026C200FBAFC6EF75F004A4FFAEF0E5C5C413136B
:0926D2005403FDE5F0EF4DFF2279
:10278C00E4F5A8F5E8F5B8F5F875650FE565A2E090
:10279C0092B5A2E192B3A2E292B4A2E392B202FF8A
:0227AC00FE220B
:10293600E565A2E092B5A2E192B3A2E292B4A2E367
:0329460092B22228
:0C29C600E5634480856482F583E0FF2215
:10002E0090D3557499F090ACAA7466F090D3557431
:10003E0090F0E562F5F0E563D2E7F583E564F582CD
:0D004E00E5F0F0E0A2E730F701B340F72243
:1024C100E565A2E092B5A2E192B3A2E292B4A2E3E1
:1024D10092B290D3557499F090ACAA7466F090D3EF
:1024E100557480F090D3557499F090ACAA7466F04D
:0924F1009080007414F0D2202246
:1029490030200D908000E020E703D38001C392205E
:03295900A2202297
:1025680075650C1224C112294940FB75650D1229A5
:1025780036E4F563F564856482856383E0F5621269
:10258800002E0564E56470020563E5647004E56384
:05259800648070E222E6
:032A5000C220227F
:03005B00021F423F
:101F4200C0E0C0D0C2CC742D25C9F5C930215015CE
:101F52004AE54A704AE54F7012854CFCC2C0F54B07
:101F6200754F01E54925E0F54A8034E54FB4011C7F
:101F720075FCFFD2C0054BE54B654D7007F54F85EB
:101F82004E4A801B754F02754A028013E54FB40218
:101F92000E854CFCC2C0754F01E54925E0F54AD0DB
:041FA200D0D0E03289
:10284F0075FCFFD2C075FE0B754C8075EA0DC2FC8E
:0D285F00D2EC754E0A7F017D011226332256
:10263300C22175FCFFD2C075FE0B8F4DE4F54F8DA3
:1026430049CEEDCEEED3940140047E3280027E0B60
:0B2653008EFE854E4AEF6002D221226D
:10295C00C22175FCFFD2C08F4EE4F54F854E4AD292
:02296C00212226
:032A53008FFE22D1
:032A56008F4C2280
:1008F9002A4D4553534147453A20615F7374203D62
:100909002025750D0A002A4D4553534147453A2084
:1009190061283029203D2025750D0A002A574152AA
:100929004E494E473A20416363656C65726174694B
:100939006F6E206F7574206F662072616E67653AFD
:1009490020615F73743D25752C2061303D2575202C
:1009590028672D7377697463682064697361626CB1
:100969006564290D0A002A4D4553534147453A20EC
:1009790070283029203D2025750D0A002A5741523B
:100989004E494E473A20507265737375726520253A
:1009990075206F7574206F662072616E6765205BC4
:1009A90025752C25755D0D0A002A5741524E494E71
:1009B900473A20427265616B776972652065727288
:1009C9006F722028425720747269676765722064C4
:1009D900697361626C6564290D0A002A5741524E98
:1009E900494E473A2049676E6974657220256264E9
:1009F90020636F6E666967757265643A20626F611C
:100A09007264206E6F7420666F756E640D0A002A19
:100A19005741524E494E473A2049676E697465728B
:100A29002025626420636F6E666967757265643A32
:100A3900206E6F20636F6E6E656374697669747971
:100A49000D0A002A5741524E494E473A20547261C5
:100A59006E736D697474657220636F6E666967750C
:100A69007265643A20626F617264206E6F742066E9
:100A79006F756E640D0A002A5741524E494E473A26
:100A89002044726F6775652069676E697465723A8B
:100A9900206E6F20636F6E6E656374697669747911
:100AA9000D0A002A5741524E494E473A204D616975
:100AB9006E2069676E697465723A206E6F20636F84
:0D0AC9006E6E65637469766974790D0A00BC
:072A0E00EF60031F80FA22B4
:10283000A20A9293E4F568F5697F78122A0E056979
:0F284000E56970020568E569640A456870EB2276
:100E7000E4906CE5F0906CE0F0A3F0906CE4F0D2BC
:100E80000A1228307F061226B2906CE1E02FF09013
:100E90006CE0E03EF0C20A122830906CE4E004F00E
:100EA000E0B420DB906CE0E0FEA3E0FF7C007D205E
:100EB00012048B906CE0EEF0A3EFF07BFF7A0879E0
:100EC000F9906CB6EEF0A3EFF01200C9E4906CE27A
:100ED000F0A3F0A3F07F061226B2906CE3E02FF0AF
:100EE000906CE2E03EF0906CE4E004F0E0B420E5C9
:100EF000906CE2E0FEA3E0FF7C007D2012048B906A
:100F00006CE2EEF0A3EFF07BFF7A09790F906CB6FC
:100F1000EEF0A3EFF01200C9906CE2E0FEA3E0FF58
:100F2000906CE0E0FCA3E0FDC39FFFEC9EFEC3EFEE
:100F3000942DEE64809480502F7BFF7A0979259060
:100F40006CB6ECF0A3EDF0906CE2E0FFA3E0906CE7
:100F5000B8CFF0A3EFF01200C97F067D041226334C
:100F6000C218906CE57406F0E4906CE0F0A3F09089
:100F70006CE4F07F071226B2906CE1E02FF0906CE9
:100F8000E0E03EF0906CE4E004F0E0B420E5906C2A
:100F9000E0E0FEA3E0FF7C007D2012048B906CE07B
:100FA000EEF0A3EFF07BFF7A09796F906CB6EEF06C
:100FB000A3EFF01200C9906CE0E0FEA3E0FFC39441
:100FC0007DEE64809482400BD3EF94DBEE648094DA
:100FD00083402E7BFF7A097985906CB6EEF0A3EF03
:100FE000F0A37402F0A3747DF0A37403F0A374DB88
:100FF000F01200C97F057D04122633906CE574055C
:07100000F0906CE5E0FF2217
:1017D400E4906CE0F0301320A294301401B340186C
:1017E4007BFF7A0979B21200C97F037D0412263384
:1017F400C213906CE07403F0E4906CE1F0906CE13F
:10180400E0FF6408606EEF25E024A2F582E4346C06
:10181400F583E0FCA3E0F47002ECF4604F1229D2EB
:1018240040217F047D041226337BFF7A0979E490FA
:101834006CE1E004906CB6F01200C9906CE07404A2
:10184400F08029906CE1E0FF12221B401F7F047D91
:10185400041226337BFF7A0A7918906CE1E0049035
:101864006CB6F01200C9906CE07404F0906CE1E086
:1018740004F08089906C91E07002A3E0601B122A4E
:101884002240167F047D041226337BFF7A0A794CAA
:0F1894001200C9906CE07404F0906CE0E0FF2249
:1024FA00D2091217D4906D32EFF06002C209120E9F
:10250A0070906D33EFF06002C20920C60B7BFF7A30
:10251A000A79801200C9C20920C70B7BFF7A0A799F
:09252A00AC1200C9C209A2092289
:10000E00E4FF742E2FF582E4346DF58374FFF00F48
:05001E00EFB404EE2226
:0C29D200EFC31325E02441FF1228A422CB
:10221B00906CE2EFF0E0FFC31325E02441FF7B015C
:10222B007A6C79E4906CE97401F0122385906CE37D
:10223B00EFF0906CE2E054012402FF74017E00C8C1
:10224B00EFC8088005C333CE33CED8F9FF906CE4CA
:0C225B00E0FDE4EF5D6003D38001C322CE
:10226700CEEFCEEEC313FF242EF582E4346DF58353
:10227700C083C082E0FDEE5401FC7401C8ECC808BD
:102287008002C333D8FCF45DD082D083F0EF25E021
:102297002440FFEEC3137C00242EF9EC346DFA7B47
:0B22A70001906CDF7401F01222FC2299
:1022B200CEEFCEEEC313FF242EF582E4346DF58308
:1022C200C083C082E0FDEE5401FC7401C8ECC80872
:1022D2008002C333D8FC4DD082D083F0EF25E024B6
:1022E20040FFEEC3137C00242EF9EC346DFA7B011F
:0A22F200906CDF7401F01222FC2250
:10200700E4F56B906C4074FFF0E4A3F0A3F0906CE0
:1020170091E0FEA3E0FFE4FCFD7BC0FAF9F81204AF
:10202700EDC8ECC8C9EDC9CAEECACBEFCB7F007EBD
:10203700C07DA87C00122341EFF404906C43F0901C
:102047006C93E0FFC43354E0FF906C9EE024182F9C
:10205700906C44F07B017A6C79407D051228F3225D
:062A22007F481228A422E7
:102120007B007C6C78077F008A838982E0B8070394
:1021300003801AB80604A31D8013F5F0A31DE8FE62
:10214000E0C5F0C5F033C5F0330EBE06F6AA83A98C
:10215000828C838B824480F0547FA3F0A3AC83AB4A
:10216000820F0FE8045407F8BD00BD221203BA9095
:092170006D34F0CFEDCFEFF02249
:1028F300122120CEEFCE7F487B017A6C7900906C59
:07290300DFEEF01222FC22BE
:10217900C0D075D008906C91E07002A3E060407403
:102189000A256BF56B906C90E0656B7032F56B907E
:102199006C4074FFF0E4A3F0A3740AF0E552A3F0D5
:1021A900E553A3F0A37401F0A304F0A304F0A3047E
:1021B900F0A304F07B017A6C79407D0A1228F3D0F0
:0221C900D02222
:1027000060206D030000CC01D8011400F0013C00F2
:102710002800E401A0016C007800B40150009C0185
:0427200088014400E8
:050026007EFF7FFF22B8
:101BD600CBEFCBCAEECAC9EDC9E9540FFFEAEB6FEA
:101BE600540F25E0FFE433FE74032FF582EE346DC7
:101BF600F583EAC4F854F0C868FEEBC4540F48FFF6
:101C0600EE540FFEE06EFAA3E06FFBCFE9CFEFC410
:101C1600540F540FFFEAEF6B540F25E0FFE433FE39
:101C260074032FF582EE346DF583EAC4F854F0C8D8
:101C360068FEEBC4540F48FFEE540FFEE06EFAA3A5
:081C4600E06FFBCEEACEFF22A5
:072A1500EEF4FEEFF4FF22D6
:10206700FF2A44FF29F2FF29FCFF27CFFF2A28FF79
:102077002725FF2A2EFF2A48FF299EFF2A34FF28FB
:1020870010FF290AFF2A4CFF2A59FF2A5AFF2A5B09
:10209700FF2A5CFF2A5DFF2A5EFF2A5FFF2A60FF97
:1020A7002A61FF2A62FF2A63FF2A64FF2A65FF2A43
:1020B7003AFF2A3AFF2A3AFF2A3AFF2A3AFF2A3AF0
:0F298F00D296D29775D8C575DBECD2BDD2AD22EA
:1028A400E4F5618F5FD222D2DDFF12265EEF641859
:0B28B4006004EFB44003D38001C32296
:1022FC00906CDCEBF0A3EAF0A3E9F0CEEFCEE4FFB8
:10230C00906CDFE06F601D906CDCE0FBA3E0FAA347
:10231C00E0F98F827583001203D3FD746C2FF8EDF6
:10232C00F60F80DC906CDFE0FFF5618E5FD222D27D
:05233C00DD12265E2207
:10238500906CE6EBF0A3EAF0A3E9F0CEEFCEA3E084
:10239500FFF5618E5FD222D2DD12265EE4FE906CDF
:1023A500E9E06E601D746C2EF8E6FD906CE6E0FBCE
:1023B500A3E0FAA3E0F98E82758300ED1204000E06
:0323C50080DC2297
:10265E00CEEFCEE4F55CEE2402FDE433FCE55C6DDA
:10266E007001EC6010755D28D55DFD202203AF6012
:0B267E0022055C80E175D8D57F0022AA
:042A440075D8D5224A
:0A29F200855FDA75D8C5E4F55E22B2
:0A29FC00855FDA75D8C5E4F55E22A8
:1027CF00C0D075D010E561700775D8D5C222800EC4
:1027DF00AF5E055E746C2FF8E6F5DA75D8C5D0D00C
:0127EF0022C7
:062A280075D8D5C2222280
:10272500C0D075D010E55E6561700775D8D5C22239
:10273500800EAF5E055E746C2FF8E6F5DA75D8C5C8
:03274500D0D022CF
:062A2E0075D8D5C222227A
:042A480075D8E52236
:0F299E00E561700775D8D5C222800375D8C522B0
:062A340075D8D5C2222274
:10281000C0D075D010AF5E055E746C2FF8A6DAE5F7
:102820005E6561700575D8C1800375D8C5D0D022AA
:10290A00C0D075D010AF5E055E746C2FF8A6DA756C
:07291A00D8D5C222D0D02263
:042A4C0075D8D52242
:012A5900225A
:012A5A002259
:012A5B002258
:012A5C002257
:012A5D002256
:012A5E002255
:012A5F002254
:012A60002253
:012A61002252
:012A62002251
:012A63002250
:012A6400224F
:012A6500224E
:062A3A0075D8D5C222226E
:03002B0002244C60
:10244C00C0E0C0F0C083C082C0D075D01085D96008
:10245C00E5D9131313541F75F003A42467F582E414
:10246C003420F583E493740193FA740293F9120502
:0C247C00BFD0D0D082D083D0F0D0E032AE
:03000000021AC71A
:0C1AC700787FE4F6D8FD7581BF021B0E8D
:1003BA00BB010689828A83E0225002E722BBFE0241
:0903CA00E32289828A83E4932274
:1003D300BB010CE58229F582E5833AF583E02250DF
:1003E30006E92582F8E622BBFE06E92582F8E22229
:0D03F300E58229F582E5833AF583E4932243
:10040000F8BB010DE58229F582E5833AF583E8F032
:10041000225006E92582C8F622BBFE05E92582C8DE
:02042000F222C6
:10042200EFF88DF0A4FFEDC5F0CEA42EFEEC88F01F
:04043200A42EFE22D4
:10043600BC000BBE0029EF8DF084FFADF022E4CCAA
:10044600F875F008EF2FFFEE33FEEC33FCEE9DEC73
:10045600984005FCEE9DFE0FD5F0E9E4CEFD22EDB9
:10046600F8F5F0EE8420D21CFEADF075F008EF2F03
:10047600FFED33FD4007985006D5F0F222C398FDF4
:050486000FD5F0EA2291
:10048B00C2D5EC30E709B2D5E4C39DFDE49CFCEE8C
:10049B0030E715B2D5E4C39FFFE49EFE120436C3CA
:1004AB00E49DFDE49CFC800312043630D507C3E4C5
:0604BB009FFFE49EFE22FB
:1004C100C5F0F8A3E028F0C5F0F8E58215827002C6
:0604D1001583E038F02263
:1004D700A3F8E0C5F025F0F0E582158270021583D8
:0604E700E0C838F0E82235
:1004ED00E88FF0A4CC8BF0A42CFCE98EF0A42CFCAE
:1004FD008AF0EDA42CFCEA8EF0A4CDA8F08BF0A42C
:10050D002DCC3825F0FDE98FF0A42CCD35F0FCEB8A
:10051D008EF0A4FEA9F0EB8FF0A4CFC5F02ECD394F
:0F052D00FEE43CFCEAA42DCE35F0FDE43CFC22BC
:10234100C2D5E830E70FB2D5E4C39BFBE49AFAE4C7
:1023510099F9E498F8EC30E717B2D5122377120611
:1023610013E4C39BFBE49AFAE499F9E498F8800337
:1023710012061330D50DE4C39FFFE49EFEE49DFDDC
:04238100E49CFC22BA
:10053C00EB9FF5F0EA9E42F0E99D42F0EC6480C836
:06054C0064809845F022D6
:10055200EB9FF5F0EA9E42F0E99D42F0E89C45F0FF
:010562002276
:10056300E8600FECC313FCED13FDEE13FEEF13FF76
:03057300D8F1229A
:0C057600ECF0A3EDF0A3EEF0A3EFF022F8
:10058200A8828583F0D083D0821205991205991230
:100592000599120599E473E493A3C583C5F0C58355
:1005A200C8C582C8F0A3C583C5F0C583C8C582C8C3
:0105B2002226
:0C05B300A42582F582E5F03583F5832253
:0605BF008A838982E473C7
:10005E00E53C24B6F582E4346CF583E0053C229051
:10006E006CB3301103906CB6E475F0011206B30256
:10007E0003BA200AE97F2ED20A8018EF540F24907B
:10008E00D43440D4FF300E0BEF24BFB41A0050030B
:10009E002461FFE53D6002153D0540E54070020517
:1000AE003F30110E906CB3E475F0011206B3EF02FF
:1000BE0005C5022A067403D2118003E4C211F53C71
:1000CE00906CB31206CAE4F53DF53FF540E53D6090
:1000DE00077F201200A180F5F53EC20BC20AC20CAA
:1000EE00C20DC20FC210C21212006DFF700D301180
:1000FE00057F001200B2AF40AE3F22B42561C2D5DB
:10010E00C20E12006DFF24D0B40A00501C75F00A06
:10011E0020D50DC53DA4253DF53D7002D20D80E0E4
:10012E00C53EA4253EF53E80D724CFB41A00EF502D
:10013E0004C2E5D20E0202ACD20B80C4D20A80BE3B
:10014E00D20C80BAD2D580B8D20F80B27F201200E6
:10015E00A1200C077401B53D0040F112005EFF12A4
:10016E0000A10200DBD212D210809312005EFB12AD
:10017E00005EFA12005EF94A4B700679787A037BBC
:10018E00FF200C33E53D602FAF3EBF00011F7E0008
:10019E008E827583001203D360050EEE6F70F1C26E
:1001AE00D5EBC0E0EAC0E0E9C0E0EE1202F0D0E02C
:1001BE00F9D0E0FAD0E0FB1203BAFF60A5EBC0E085
:1001CE00EAC0E0E9C0E01200A1D0E02401F9D0E0DD
:1001DE003400FAD0E0FBE53E60DDD53EDA80837B6D
:1001EE00FF7A0279ECD20C8098791080027908C2DD
:1001FE0010C2128008D2D5790A8004790AC2D5E4D9
:10020E00FAFDFEFF12005EFC7B08200B1312005E4F
:10021E00FD7B10300A0A12005EFE12005EFF7B208C
:10022E00EC3382D592D55013C3E4300A069FFFE417
:10023E009EFEE4200B039DFDE49CFCE4CBF8C20B78
:10024E00EC700CCFCECDCCE824F8F870F38017C349
:10025E00EF33FFEE33FEED33FDEC33FCEB33FB9966
:10026E004002FB0FD8E9EB300B05F8D0E0C448B2E2
:10027E000BC0E00AEC4D4E4F78207B0070C2EAC0F6
:10028E00E01202F2D0F0D0E0200B04C4C0E0C4B201
:10029E000BC0F012008AD0F0D5F0EB0200DB120694
:1002AE00D301795301F758014A4C01464201FB4FE5
:1002BE00020344020349015F4302095501ED460161
:1002CE00ED4501ED47039B50014E2D01522E017558
:1002DE002B01562301732003862A0000016D3F3F38
:1002EE003F00790AA2D5200D14300F09B91002046F
:1002FE0004B9080104A2D5201002500104200C6696
:02030E00920C4F
:10031000B53D005032C0E07F20300D177F30A20C79
:100320007210720F500D120347C20CC210C20F7F21
:1003300030800F300F03E9C0E01200A1300F03D06E
:10034000E0F9D0E0B53DCE300F177F30B9100C1278
:1003500000A17F58300E077F788003B90803120090
:10036000A1300C057F2D0200A17F202012F87F2BE9
:100370002010F322920C80CF286E756C6C29002D12
:1003800050434958D20B12005E300BF8C20B783D37
:1003900030D504D20A783EF602010C12005E240326
:1003A000B405004001E490037F93120092743A1266
:0A03B0000092D20D753D040201F722
:10292100EFC394094006EFC3940E4004EFB42003B3
:05293100D38001C32268
:101E7500906CE0EBF0A3EAF0A3E9F0906CE3E0FBF3
:101E8500A3E0FAA3E0F91203BAFE906CE0E0FBA32D
:101E9500E0FAA3E0F91203BAFD6E702AED600E9028
:101EA5006CE674FFF5F01204C145F070037F002263
:101EB500906CE1E475F0011204C1906CE4E475F0F6
:101EC500011204C180B5D3EE6480F8ED64809840BA
:071ED500037F01227FFF22C1
:10288800E94A4B7001221203BAFF6D700122EF7002
:0C28980004FBFAF92209E970ED0A80EA5D
:1012F300906CF1EBF0A3EAF0A3E9F0906CF1E0FB62
:10130300A3E0FAA3E0F91203BAFF122921500C90CB
:101313006CF2E475F0011204C180E0D209906CF123
:10132300E0FBA3E0FAA3E0F91203BAFF642B600425
:10133300EFB42D1D906CF1E0FBA3E475F0011204F2
:10134300D7A9F0FA1203BA642D6003D38001C392C4
:1013530009906CF412058200000000906CF1E0FB30
:10136300A3E0FAA3E0F91203BAFF12296E506A7FD1
:101373000A7E007D007C00906CF4E0F8A3E0F9A302
:10138300E0FAA3E0FB1204EDC8ECC8EDC0E0EEC048
:10139300E0EFC0E0906CF1E0FBA3E0FAA3E0F91208
:1013A30003BAFF3395E0FEEF24D0FFEE34FFFEE4F3
:1013B300FCFDD0E0FBD0E0FAD0E0F9EB2FFFEA3EF2
:1013C300FEED39FDEC38FC906CF4120576906CF26E
:1013D300E475F0011204C18082300910906CF4E0CE
:1013E300FCA3E0FDA3E0FEA3E0FF8011906CF4E01A
:0E13F300FCA3E0FDA3E0FEA3E0FF1206A5228E
:1016FC00906CFEEBF0A3EAF0A3E9F0906CFEE0FB3B
:10170C00A3E0FAA3E0F91203BAFF122921500C90BE
:10171C006CFFE475F0011204C180E0D209906CFEFC
:10172C00E0FBA3E0FAA3E0F91203BAFF642B600418
:10173C00EFB42D1D906CFEE0FBA3E475F0011204D8
:10174C00D7A9F0FA1203BA642D6003D38001C392B7
:10175C0009E4906D01F0A3F0906CFEE0FBA3E0FABD
:10176C00A3E0F91203BAFF12296E503F906CFEE011
:10177C00FBA3E0FAA3E0F91203BAFF3395E0FEEF06
:10178C0024D0FBEE34FFFA906D01E0FEA3E0FF7C69
:10179C00007D0A120422EF2BF0EE3A906D01F090CE
:1017AC006CFFE475F0011204C180AD30090A906D34
:1017BC0001E0FEA3E0FF800F906D01E0FEA3E0FFCF
:0817CC00C3E49FFFE49EFE222E
:101AD300021CC1E493A3F8E493A34003F68001F24C
:101AE30008DFF48029E493A3F85407240CC8C33314
:101AF300C4540F4420C8834004F456800146F6DFE3
:101B0300E4800B0102040810204080902700E47E4B
:101B1300019360BCA3FF543F30E509541FFEE493D7
:101B2300A360010ECF54C025E060A840B8E493A39E
:101B3300FAE493A3F8E493A3C8C582C8CAC583CAC9
:101B4300F0A3C8C582C8CAC583CADFE9DEE780BE81
:0127240000B4
:1005C500BB010689828A83F0225002F722BBFE0115
:0205D500F3220F
:1005D70075F008758200EF2FFFEE33FECD33CDCCDB
:1005E70033CCC58233C5829BED9AEC99E58298405E
:1005F7000CF582EE9BFEED9AFDEC99FC0FD5F0D63B
:10060700E4CEFBE4CDFAE4CCF9A88222B800C1B964
:100617000059BA002DEC8BF084CFCECDFCE5F0CBA2
:10062700F97818EF2FFFEE33FEED33FDEC33FCEBDB
:1006370033FB10D703994004EB99FB0FD8E5E4F996
:10064700FA227818EF2FFFEE33FEED33FDEC33FC83
:10065700C933C910D7059BE99A4007EC9BFCE99A77
:10066700F90FD8E0E4C9FAE4CCFB2275F010EF2FBC
:10067700FFEE33FEED33FDCC33CCC833C810D707BC
:100687009BEC9AE899400AED9BFDEC9AFCE899F8F7
:0E0697000FD5F0DAE4CDFBE4CCFAE4C8F9228A
:0E06A500C3E49FFFE49EFEE49DFDE49CFC2266
:1006B300F8E0FBA3A3E0F925F0F0E58215827002D0
:0706C3001583E0FA38F02274
:0906CA00EBF0A3EAF0A3E9F02231
:1006D300D083D082F8E4937012740193700DA3A3B6
:1006E30093F8740193F5828883E4737402936860CA
:0606F300EFA3A3A380DFCA
:10296E00EFC394304009EFC3943A5003D38001C3B0
:01297E002236
:00000001FF
